:020000040000FA
:060000008A150A16612DAD
:043000000034003464
:1038000083120313FB308605083086041030BE0097
:1038100020308400B02580003C302002031D0A2C9B
:10382000840ABE0B0A2CC3010C30BE002130840078
:103830000008C307840ABE0B182C0A30BE002530CE
:1038400084000008C1258000840ABE0B212C2808B2
:10385000B900270EB9042608B800250EB8042C08B4
:10386000BD002B0EBD042A08BC00290EBC0438087C
:10387000BA003908BB003D08BB07031C402CBA0A3C
:103880003C08BA073C302002031DBB2C3E302F02FF
:10389000031DBB2C2E08F5002D0EF5044308750200
:1038A000031DBE2C1B303A020319592C031C602C3B
:1038B000C12CFF303B020319602C0318C12C602C73
:1038C000003038020319672C03186D2CC12C04300A
:1038D000390203196D2C031CC12CC724B025A0008C
:1038E0007B302002031DBB2CC3013808F4003908CB
:1038F000F300F501F6010430BE0020308400B0254D
:10390000C307C1258000840ABE0B7F2C2308F60064
:10391000220EF6042108F500200EF504FF24000015
:103920000000000000000000000000000000000097
:10393000F30A0319F40A3A087402031D792C3B08B0
:103940007302031D792CB025C125A000B025C12527
:10395000A100200EA10443082102031DBE2CB025A6
:10396000A0007D302002031DBB2C83120313F7300F
:103970008605C724BA2C3130D824692D3430D82498
:10398000692D3630D824692D3730D824692D5B3025
:10399000AA253030AA253830AA253130AA25303062
:1039A000AA254330AA253930AA255D30AA2508006A
:1039B000F500B025A0007D3020020319E42C3E3034
:1039C00020020319E42CD92C5B30AA253030AA251B
:1039D0004130AA253030AA253030AA253030AA251A
:1039E0007508AA253330AA25750AAA255D30AA25AF
:1039F00083120313F730860504308604080003178A
:103A0000831273088D0074088F0075088C00760887
:103A10008E0083168C170C158B1355308D00AA3031
:103A20008D008C14000000000C1103138312080099
:103A30000317831273088D0074088F0083168C1788
:103A40000C140000000083120C08F7000E08F800A8
:103A5000031308008312031386168316403099005F
:103A6000243098008312903098001A081A087010B9
:103A70000800831203138C1A472D81010B11861243
:103A80008C1A472D7018402D0B1D402D492D1A08FA
:103A9000512D18194F2D98184F2D0301512D181223
:103AA00018168616BF01BF0B532DBF010800031364
:103AB0008312061A592D8316981C5C2D83129900C7
:103AC000080083120313D1256625692D2A25E925CF
:103AD00008007010B025F900553079020319812DC6
:103AE000563079020319922D5A3079020319962D16
:103AF000503079020319A42D463079020319A72DFD
:103B0000692D7014F01C852D872D18128A2D8316AF
:103B1000091283128312031306117530AA258A0134
:103B20001030820070147630AA25002C7014831295
:103B3000031306110130AA250130AA250130AA2558
:103B40000330AA257010692D86150611A62D0615BD
:103B50008611A92DF01CAE2D5725AF2D0526080086
:103B6000701CB92DF01CB72DB52D3925C02DF125B0
:103B7000C02DF018BC2DBE2DF010B72DF014B52DB2
:103B80000800FA00F9000F30F90547307A020318EF
:103B9000CF2D41307A02031CCF2D0930F907790867
:103BA0000800031383160B30850010308600903018
:103BB00087001730890004309F008312033087008C
:103BC00000308600103085008316D63081008312C5
:103BD000080003138316173089008312031306109D
:103BE0000800831203133D3081000B110614831665
:103BF000891B002E7018F72D0B1DF72D0301032EC6
:103C000083120610080806100800831203138800A8
:0E3C100006148316091B0A2E831206100800E4
:02400E003A3F37
:00000001FF
